:0514E500323732430024
:1013D700AF8475840F75E10343E20443E3C075A44A
:1013E7000F7580F075A50775AD0775A6FF75A0FF8A
:0513F70075A7E08F84E2
:0113FC0022CE
:10148600AF84E4F584759D0443F808759A40D2F854
:021496008F8441
:011498002231
:0614DA00121459021486F1
:0514E0001213D7D32216
:1012F700C200C201C20275FFDE75FFAD1214E09293
:101307000030005A1214DA7BFF7A1479E5120DEED9
:10131700EF24FF92013001127D007C08E4FFFE12EA
:1013270013B0E4FFFE120F2C80217BFF7A1479E5BE
:10133700121067EF24FF92023002107D007C08E450
:10134700FFFE1213B0E4FFFE120C1AE4FFFE0FBFFC
:1013570000010EBE27F8BF10F5E4F584F5C080FE46
:101499002321323030454655002324323030454629
:0214A9005500EC
:10145900AF8475840F758A83E4F597F58475C04464
:0714690075CFE4C2C38F84BC
:011470002259
:06141F008F27AD27AF2668
:021425008D1E1A
:101427001213FDEFC454F0F51FAF1E1213FDEF2585
:041437001FF51FFF7F
:01143B00228E
:1013B0008F828E83D3E5829DE5839C501943B701CC
:1013C000758F03E4F0F58F53B7FE2582F582740420
:0613D0003583F58380DE89
:0113D60022F4
:02118800A907B5
:10118A0020C3FD20C5FAC2C4D2C5E4FFFC30C3FDAA
:10119A0030C3FDE5C154F8FA64086003BA1011E5DA
:1011AA001DBF01044401800254FEF5C27C01807C0B
:1011BA00BA180B851CC27C02C2C4C2C5806EBA2092
:1011CA00028038EA64287030B9010CBC020280152A
:1011DA00EC6404701F8019BC02088BC27C03C2C570
:1011EA008012BC03088DC27C04C2C58007BC0404FB
:1011FA00D2C57F01C2C48034BA300AD2C4D2C57CF7
:10120A0009E4FF8027BA3802801EBA4006C2C2C269
:10121A00C58019BA48028010BA50028003BA580829
:10122A00D2C47C08AEC28004D2C4D2C5C2C3EC64A4
:08123A0008600302119AAF06DF
:011242002289
:1014BC00AE05AD078E1C8B1DE4FB7F01121188223B
:1014AB00AE03AB05AD078E1C751DA07F0212118814
:0114BB00220E
:060DEE008B3D8A3E893FA7
:100DF4007547FF7548147549997544017545007523
:100E04004600E4F543F542F541F540E47F50FEFD2C
:100E1400FCAB43AA42A941A840C312129B5036AF6F
:100E2400437BA0E4FD1214BCAB440546E546AA4549
:100E34007002054514F9EF121289E4FAF9F8E54352
:100E44002401F543EA3542F542E93541F541E835F7
:100E540040F54080B6AB47AA48A949121243FF9017
:100E64000000E06F706290000112125CFF900001BC
:100E7400E06F705490000212125CFF900002E06F69
:100E8400704690000312125CFF900003E06F70380C
:100E940090000412125CFF900004E06F702A90002E
:100EA4000512125CFF900005E0B5071C90000612C5
:100EB400125CFF900006E0B5070E90000712125C6A
:100EC400FF900007E06F60037F0022AB3DAA3EA9BC
:100ED4003F121243FF900011E06F702A900001123C
:100EE400125CFF900012E0B5071C90000212125C25
:100EF400FF900013E0B5070E90000312125CFF9000
:100F04000014E06F60037F0022900009E0F55BA30A
:100F1400E0F55DA3E0F55E900019E0F557A3E0F578
:070F240059A3E0F55A7F011B
:010F2B0022A3
:0D143C008F0DAF18AE171214718E178F1898
:02144900AC06EF
:0D144B00AB07AF04AD07AF03AB581214BCE4
:011458002271
:0E14CC00E55CC3955B500605580558055C228B
:101471000FBF00010ED3EF955EEE955D400612148D
:05148100CCE4FEFF2297
:040F2C008E088F0993
:100F3000E4F50DF50EF513F514F515F516F517F5A1
:100F400018855917855A18855758F50EF50D755C93
:100F500001E4F512E50D643A6016AF18AE171214ED
:100F6000498F0DAF18AE171214718E178F1880E4C9
:100F70000514E51470020513AF18AE1712144912C8
:100F8000143C8F0EAD0EAF0D1214258F108510126C
:100F900012143E12143C8F0EAD0EAF0D12142575B7
:100FA00015008F16EF2512F512E516751600F515CA
:100FB00012143E12143C8F0EAD0EAF0D121425EF1D
:100FC000421685150A85160BE5162512F512121420
:100FD0003E12143C8F0EAD0EAF0D1214258F0FE58F
:100FE0000F2512F512E50F705CF50CE50CC395109A
:100FF000505312143E12143C8F0EAD0EAF0D12144E
:10100000258F11E5112512F512C3E50B9509E50AA7
:101010009508402DAE0AAF0BBEFB06BFFE0343B1E1
:101020003043B701758F01850B82850A83E511F086
:10103000E4F58F53B7FE75B111050BE50B70020592
:101040000A050C80A612143E12143C8F0EAD0EAF92
:101050000D1214258F11E5112512700AE50F640198
:061060006003020F5122A3
:011066002267
:061067008B4A8A4B894C04
:10106D007554FF7555147556A2755101755200755D
:10107D005350E4F550F54FF54EF54DE47F2BFEFD45
:10108D00FCAB50AA4FA94EA84DC312129B5035AFC1
:10109D0050E4FBFD1214ABAB510553E553AA52704E
:1010AD0002055214F9EF121289E4FAF9F8E5502409
:1010BD0001F550EA354FF54FE9354EF54EE8354D12
:1010CD00F54D80B7AB54AA55A956121243FF9000A7
:1010DD0050E06F706290000112125CFF900051E0C1
:1010ED006F705490000212125CFF900052E06F700E
:1010FD004690000312125CFF900053E06F70389021
:10110D00000412125CFF900054E06F702A900005ED
:10111D0012125CFF900055E0B5071C9000061212EC
:10112D005CFF900056E0B5070E90000712125CFFB1
:10113D00900057E06F60037F0022AB4AAA4BA94C89
:10114D00121243FF90005FE06F702A90000112129F
:10115D005CFF900060E0B5071C90000212125CFF6E
:10116D00900061E0B5070E90000312125CFF900035
:0A117D0062E06F60037F00227F0133
:011187002245
:10136700E48F34F533F532F531AE33AD32AC317845
:10137700081212C48F348E338D328C3178351212A5
:01138700D78E
:081388008F628E618D608C5FA5
:10139000AA0778081212B1A907AF62AE61AD60ACBE
:0F13A0005F78101212B1AB07AF02AD011214ABA0
:0113AF00221B
:040C1A008E218F2276
:100C1E00E4F526F527F534F533F532F531F538F5EB
:100C2E0037F536F535F53CF53BF53AF53975382B94
:100C3E00F537F536F535F527F526F52CE4F52BE5E4
:100C4E0026643A60071213838F2680F3E53C240155
:100C5E00F53CE4353BF53BE4353AF53AE43539F508
:100C6E00391213838F2612138312141F8F2985298D
:100C7E002B1213838F2612138312141FE48F30F559
:100C8E002FF52EF52DEF252BF52BAE2FAD2EAC2DF2
:100C9E0078081212C48F308E2F8D2E8C2D12138346
:100CAE008F2612138312141FE5304FF530E52FF502
:100CBE002FE52EF52EE52DF52D852F23853024E5F8
:100CCE0030252BF52B1213838F2612138312141F2C
:100CDE008F28E528252BF52BE5286404703B12138D
:100CEE00838F2612138312141F1213678F2612136B
:100CFE008312141FE5344FF534E533F533E532F541
:100D0E0032E531F531AF34AE33AD32FC781012121C
:100D1E00C48F348E338D328C31E5286402703B12D1
:100D2E0013838F2612138312141F1213678F26122A
:100D3E00138312141FE5344FF534E533F533E532E2
:100D4E00F532E531F531AF34AE33AD32FC78041205
:100D5E0012C48F348E338D328C31E5342524F52434
:100D6E00E5333523F523E5287058F525E525C3959C
:100D7E0029504F1213838F2612138312141F8F2A9A
:100D8E00E52A252BF52BC3E5249522E52395214055
:100D9E002DAE23AF24BEFB06BFFE0343B13043B7D7
:100DAE0001758F01852482852383E52AF0E4F58F72
:100DBE0053B7FE75B1110524E524700205230525F0
:100DCE0080AA1213838F2612138312141F8F2AE503
:0F0DDE002A252B700AE52864016003020C4A22C3
:010DED0022E3
:03000000020C00EF
:03000300021A03DB
:03000B00021A06D0
:03001300021A09C5
:03001B00021A0CBA
:03002300021A0FAF
:03002B00021A12A4
:03003300021A1599
:03003B00021A188E
:03004300021A1B83
:03004B00021A1E78
:03005300021A216D
:03005B00021A2462
:03006300021A2757
:03006B00021A2A4C
:03007300021A2D41
:03007B00021A3036
:03008300021A332B
:03008B00021A3620
:03009300021A3915
:03009B00021A3C0A
:0300A300021A3FFF
:100C0000787FE4F6D8FD9000007F007E20E4F0A31A
:0A0C1000DFFCDEFA7581620212F7C4
:10124300BB010689828A83E0225002E722BBFE02A9
:09125300E32289828A83E49322DC
:10125C00BB010CE58229F582E5833AF583E0225047
:10126C0006E92582F8E622BBFE06E92582F8E22291
:0D127C00E58229F582E5833AF583E49322AB
:10128900BB010689828A83F0225002F722BBFE0144
:02129900F3223E
:10129B00EB9FF5F0EA9E42F0E99D42F0EC6480C8CA
:0612AB0064809845F0226A
:1012B100E8600FECC313FCED13FDEE13FEEF13FF1B
:0312C100D8F1223F
:1012C400E8600FEFC333FFEE33FEED33FDEC33FC88
:0312D400D8F1222C
:1012D7007401FF3395E0FEFDFC080808E6CF2FF602
:1012E70018E6CE3EF618E6CD3DF618E6CC3CF622DB
:1013FD00EF7E0024D0B40A00401624F9B40A004050
:10140D000CB41000400A24E0B41000400374FFFE39
:02141D00FF22AC
:00000001FF
